:1000000000308A008A280000FF00030E8301A1004F
:100010007F08A0000A08A8008A01A00E0408A20018
:100020007708A3007808A4007908A5007A08A6003C
:100030007B08A700831383128C308400001C2228C5
:100040000C183528220884002308F7002408F8003B
:100050002508F9002608FA002708FB0028088A006E
:10006000210E8300FF0E7F0E09008A11372885308C
:100070008F00ED308E002A082902031C52288316B7
:100080000C1083122D10051483160510831286128E
:10009000861386108510831685108312051183162A
:1000A00005118312A90A0C108A1122282F3084000E
:1000B00083130008031962285230F700F70B5E28FB
:1000C000800B5C28003486108612861385148316F4
:1000D00085108312051583160511831205148316E6
:1000E000051002308312AE00FA30AF005620AE0B7E
:1000F0007428851083168510831205118316051147
:100100008312051083160510FA308312AF005620B3
:100110008A11AD28840183131F3083054230831672
:100120008F000F081F129F121B0880399B00073099
:100130009C008312A901AA010530AB000A30AC0073
:100140002D10403083168F000F0818308500513075
:100150008600B53083129000632883160C10C030DF
:1001600083128B042D180C2906180C290A30AA00BA
:10017000A9018316851583128519C0282B08AA07A3
:10018000831605168312051AC7282C08AA07061F0E
:100190000C292D1486128617861405108316051057
:1001A0008312851083168510831205158316051199
:1001B0000C14831286160230AE00FA30AF005620BF
:1001C000AE0BDD2886122D1CEF28061AEF28051528
:1001D0008316051132308312AF005620E3282D1C00
:1001E0000C29061E0C292D1083160C1083122A08C8
:1001F00029020318FF2885148316851083120830FE
:10020000AE00FA30AF005620AE0B012986138610DF
:100210000511831605118312061B2D292D10861337
:10022000861286100510831605108312851083161A
:100230008510831205118316051183128612851409
:100240008316851064308312AF0056208510831604
:0E025000851064308312AF005620B228630080
:04400E00103FFF3F21
:00000001FF
